:100000000C9404030C943C030C943C030C943C03AC
:100010000C943C030C943C030C943C030C943C0364
:100020000C943C030C943C030C9499260C946B2781
:100030000C9478210C943C030C943C030C943C03EA
:100040000C943C030C943C030C943C030C943C0334
:100050000C943C030C9400220C943C030C943C0341
:100060000C943C030C943C030C943C030C943C0314
:100070000C943C030C943C030C943C030C943C0304
:100080000C943C030C943C030C943C030C943C03F4
:100090000C943C030C943C030C943C030C943C03E4
:1000A0000C943C030C943C030C943C030B060B0691
:1000B000370637069F06BD06D507D507C806610770
:1000C00072077207D827FF27F728FF27F7284B2842
:1000D0006E28F728C528D42829001E001F002000FC
:1000E00021002200230024002500260027002D00E7
:1000F0002E0000002A002B0014001A000800150032
:1001000017001C0018000C00120013002F00300014
:1001100031000000390004001600070009000A0041
:100120000B000D000E000F0033003400000028000B
:100130000000E10000001D001B0006001900050082
:10014000110010003600370038000000E500000004
:10015000E000E300E2002C00E600E7000151E400CB
:1001600059005A005B005800620063000000000064
:1001700000000000000000000000000000005F0020
:100180006000610057005C005D005E000000000040
:1001900000000000000000000000000053005400B8
:1001A0005500560000000000000035003A003B00FA
:1001B0003C003D003E003F00400041004200430043
:1001C0004400450000004C00010001005200010005
:1001D000005C010001000100010001004600470031
:1001E0004800010000000100500051004F000100D4
:1001F000010001000100010049004A004B0000001D
:100200000100000001000000AA00A900A800C35CD2
:10021000C55CC45CCB5CCA5C4D004E0000000100B4
:1002200000000100010001000100010001000100C7
:1002300001000100010001000100010001000000B7
:1002400000000000000000000000000000000000AE
:100250000100010001000100010001000100000097
:10026000000000000000000000000000000001008D
:1002700001000100010000000000000000047F3FB9
:100280001F643214643214783C1E1E140A052223A3
:10029000252628292A2C2D2F3032333536383A3B63
:1002A0003D3E4042434547494A4C4E5051535557B5
:1002B000595A5C5E6062646668696B6D6F717375D4
:1002C00077797B7D7F81838587898A8C8E909294D4
:1002D00096989A9C9E9FA1A3A5A7A8AAACAEAFB1E1
:1002E000B3B4B6B8B9BBBCBEBFC1C2C3C5C6C7C92B
:1002F000CACBCCCDCED0D1D2D2D3D4D5D6D7D7D8E5
:10030000D9D9DADADBDBDBDCDCDCDCDCDDDDDDDD36
:10031000DCDCDCDCDCDBDBDBDADAD9D9D8D7D7D63E
:10032000D5D4D3D2D2D1D0CECDCCCBCAC9C7C6C5F5
:10033000C3C2C1BFBEBCBBB9B8B6B4B3B1AFAEAC3B
:10034000AAA8A7A5A3A19F9E9C9A98969492908EE6
:100350008C8A89878583817F7D7B79777573716FBF
:100360006D6B6968666462605E5C5A59575553519B
:10037000504E4C4A4947454342403E3D3B3A383651
:10038000353332302F2D2C2A292826252322FFAA67
:100390007F5540000101010101010101010202023A
:1003A0000202020202020303030303030303040421
:1003B00004040404040505050505060606060607EB
:1003C0000707070708080808090909090A0A0A0BA4
:1003D0000B0B0C0C0C0D0D0D0E0E0E0F0F0F101045
:1003E00011111112121313141415151616171718CC
:1003F0001819191A1A1B1B1C1D1D1E1E1F20202137
:100400002222232424252626272829292A2B2C2D7D
:100410002D2E2F30313232333435363738393A3B9E
:100420003C3D3E3F404142434445464748494A4C93
:100430004D4E4F50515354555658595A5B5D5E5F5F
:10044000616264656668696B6C6D6F7072737577F5
:10045000787A7B7D7E8082838587888A8C8E8F9157
:10046000939596989A9C9EA0A2A3A5A7A9ABADAF81
:10047000B1B3B5B7BABCBEC0C2C4C6C9CBCDCFD16B
:10048000D4D6D8DBDDDFE2E4E7E9EBEEF0F3F5F814
:10049000FAFDFF10034C002B004D00200036003009
:1004A000004E0000001A034C002B004D0020004BB2
:1004B000006500790062006F006100720064000056
:1004C000000403090409023B00020100A0FA090428
:1004D0000000010301010009211101000122400077
:1004E0000705810308000109040100010300000061
:1004F00009211101000122B6000705820320000135
:1005000012010002000000084D4C014B01000102E5
:10051000000105010902A10185020901A1000509E7
:1005200019012908150025019508750181020501A9
:10053000093009311581257F950275088106093832
:100540001581257F950175088106050C0A3802156D
:1005500081257F950175088106C0C005010980A12C
:1005600001850319012AB700150126B70095017509
:10057000108100C0050C0901A101850419012AA000
:1005800002150126A002950175108100C005010920
:1005900006A1018506050719E029E7150025019543
:1005A00008750181020507190029EF15002501953D
:1005B000F07501810205081901290595057501915C
:1005C00002950175039101C005010906A101050706
:1005D00019E029E7150025019508750181029501AB
:1005E000750881010507190029FF150026FF0095F0
:1005F0000675088100050819012905950575019101
:1006000002950175039101C011241FBECFEFDAE0FE
:10061000DEBFCDBF04B603FE18C08091AD0390913C
:10062000AE03A091AF03B091B0038730904BA740C9
:10063000B04B59F41092AD031092AE031092AF0379
:100640001092B003E0E0F8E3099511E0A0E0B1E01A
:10065000E4E5F4E502C005900D92AA3CB107D9F794
:1006600023E0AAECB1E001C01D92AD3AB207E1F778
:100670000E94E1130C94282A0C94000081E0089554
:1006800081E008950C94400308950C9444031F9353
:10069000CF93DF9300D000D01F92CDB7DEB7498350
:1006A0005A836B833091CD0189819A81311114C0B5
:1006B000662359F0222349F00E94120A182F682F4E
:1006C00089819A810E94BB0903C00E94E609182F04
:1006D00069817A81812F04C00E94120A69817A811E
:1006E0000F900F900F900F900F90DF91CF911F916F
:1006F0000C944C11FC01262F408151816281738141
:1007000084810C94470381E00895CF93DF93EC013B
:1007100060E00E947A03BE01DF91CF910C94450303
:100720000C9492120C948E1208950E9465080E94F7
:1007300094032FEF84E39CE0215080409040E1F748
:1007400000C000000C9426220F931F93CF93DF93D9
:100750008C0161E00E947A03EC01B8010E9442031F
:10076000882309F444C0B801CE010E94C31F882326
:10077000F1F1B801CE010E94D71D8823C1F1B80163
:10078000CE010E941F1F882391F1B801CE010E9463
:10079000DD1C882361F1F8018281882309F1CB35C2
:1007A0008DE5D807C1F050F4C115FCE5DF0781F0F5
:1007B000CF3DDC45A9F40E94490F19C0CC35EDE5C9
:1007C000DE0761F0CD35DD4559F40E948C0E08C07E
:1007D0000E9495030CC00E94950E02C00E94980EC4
:1007E000C801DF91CF911F910F910C943E0380E0DF
:1007F000DF91CF911F910F9108950E945A210E947D
:100800002E040C945A1B0E9431040E94261C0C9446
:10081000602108950C94090481E00895CF93C82FB6
:100820000E940C04882351F0C0FF02C02F9A01C01F
:100830002F98C1FF02C0479A01C04798CF910895F1
:10084000279A2F983F9A47980895CF93C82F0E94D0
:100850000A048C2F0E940E04CF91089580E00C941E
:1008600025040E941F200C9425040E941F209091B3
:10087000CC01891721F08093CC010C9425040895B4
:10088000CF93DF93CDB7DEB72B970FB6F894DEBFCB
:100890000FBECDBF4F83588769877A878B876111D9
:1008A0000E94D80D9E012F5F3F4F86E0F901119203
:1008B0008A95E9F785E0FE013796D90101900D92FE
:1008C0008A95E1F789819A814C815D81452B31F0D0
:1008D0009F3F31F491E08F3F19F403C091E001C0D4
:1008E00090E090FF09C049815A816B817C818D81A4
:1008F0009E810E94F90C05C0C9010E9483038111E9
:10090000F2CF2B960FB6F894DEBF0FBECDBFDF91AE
:10091000CF910895FC01808191810E94540A08952D
:10092000CF93882309F4A4C0C82F8238C1F40E9451
:100930001F2081FD9DC069E3809102019091030118
:100940000E9415210E94FA0D2FEF81EE94E02150B4
:1009500080409040E1F700C0000069E319C083388F
:1009600001F50E941F2080FD83C063E58091020194
:10097000909103010E9415210E94FA0D2FEF81EE44
:1009800094E0215080409040E1F700C0000063E512
:1009900080910201909103010E942021CF910C943B
:1009A000FA0D8438C1F40E941F2082FD61C067E403
:1009B00080910201909103010E9415210E94FA0D7D
:1009C0002FEF81EE94E0215080409040E1F700C08D
:1009D000000067E4DDCF8CEF8C0F813AD0F46C2FF0
:1009E00080910201909103010E949520882349F093
:1009F0006C2F80910201909103010E9420210E949E
:100A0000FA0D6C2F80910201909103010E94152133
:100A1000C5CF80E28C0F883048F4C77081E001C0F8
:100A2000880FCA95EAF70E94BB0DB8CFEBE5EC0F33
:100A3000E33040F4F0E0E65AFE4F808190E0CF9141
:100A40000C945320E8E5EC0FE73150F4F0E0EE0FA2
:100A5000FF1FE45DFE4F80819181CF910C9469204E
:100A6000CD3E30F08C2F0E946614CF910C94381537
:100A7000CF910895882309F464C0823879F40E94E4
:100A80001F2081FF5EC069E3809102019091030104
:100A90000E9415210E94FA0D69E310C08338B1F459
:100AA0000E941F2080FF4DC063E58091020190915C
:100AB00003010E9415210E94FA0D63E58091020155
:100AC000909103010E9420210C94FA0D843879F44E
:100AD0000E941F2082FF35C067E48091020190913F
:100AE00003010E9415210E94FA0D67E4E7CF9CEFF5
:100AF000980F913A10F4682FE1CF90E2980F983058
:100B000050F4877091E001C0990F8A95EAF7892F18
:100B10000E94C10DD9CF9BE5980F933020F480E05F
:100B200090E00C94532098E5980F973120F480E0E2
:100B300090E00C9469208D3E20F00E94C1140C942A
:100B4000381508951F93CF93DF93182FEB010E9460
:100B50009004209741F08FE99FE00197F1F700C0E2
:100B600000002197F6CF812FDF91CF911F910C9438
:100B70003A05893319F060E070E002C060E570E08A
:100B80000C94A205882321F00E94BB0D0C94FA0D51
:100B90000895882321F00E94C10D0C94FA0D089548
:100BA000CF92DF92EF92FF920F931F93CF93DF9339
:100BB0007C01D62FC72FFC011281058102950F7091
:100BC0000E94B10D8823B9F01123A9F08C2F807FEA
:100BD000803421F080E28D0F883068F08091FF0230
:100BE00082FD09C082E00E945A0E0E94B10D91E080
:100BF000D82ED92601C0D12CCC2EC2948FE0C82289
:100C00008C2D90E08C30910508F0CFC1FC01EA5AA0
:100C1000FF4F0C9483298C2F807FCF70882311F095
:100C2000C295C07F112399F0CC2309F4AAC180E2B8
:100C30008D0F883010F0D11104C08C2F0E94BB0D95
:100C400003C08C2F0E94CB0D0E94FA0D9AC18D2FEC
:100C50000E943A05CC2309F4A8C180E28D0F8830A8
:100C600038F1DD2329F18C2F0E94D10D24C08C2F67
:100C7000807FCF70803211F0C295C07FDD2319F0E4
:100C8000D130A1F13DC08091FF0282FF17C0112336
:100C900049F0CC2329F08C2F0E94BB0D0E94FA0D45
:100CA00080E070C180E00E943A05CC2309F47DC148
:100CB0008C2F0E94C10D0E94FA0D77C1112371F093
:100CC000002341F0013031F40E94DB0D8C2B0E9497
:100CD000E30D6BC10E94DB0D8C2B1DC0002319F0AE
:100CE000013009F462C10E94F00D25C0112321F0EA
:100CF000063008F05AC10EC0053008F056C11BC0BE
:100D0000112361F0002331F0F701858180FF39C1A3
:100D10008F7085838C2F0E94C20547C1002359F034
:100D2000D93309F03FC1FFEF07EE13E0F150004067
:100D30001040E1F735C18C2F0E94C90536C18C2FB8
:100D400086958695837019F0813061F02EC111234C
:100D500021F08D2F9C2F937002C080E090E00E94C4
:100D600053202BC1112321F08D2F9C2F937002C093
:100D700080E090E00E94692020C18D2F112319F09E
:100D80000E94661402C00E94C1140E94381515C149
:100D90008C2F837009F047C011110BC12D2F2295A4
:100DA00026952770220F220F6D2F6F70862F90E0EF
:100DB000A0E0B0E0022E04C0880F991FAA1FBB1F3D
:100DC0000A94D2F7D4FF10C04FE050E060E070E02A
:100DD00004C0440F551F661F771F2A95D2F7409510
:100DE00050956095709503C040E050E0BA01C695FB
:100DF000C695C3708A019B01082B192B2A2B3B2B0C
:100E0000C901B801C23049F058F4C13019F00E944C
:100E1000D108CFC00E94BF08CCC00E94E308C9C05F
:100E20000E94BD08C6C0112319F08C2F817001C02B
:100E30008695882309F4BDC02D2F2295269527700D
:100E4000220F220F6D2F6F70862F90E0A0E0B0E090
:100E5000022E04C0880F991FAA1FBB1F0A94D2F745
:100E6000D4FF10C04FE050E060E070E004C0440FD9
:100E7000551F661F771F2A95D2F7409550956095AC
:100E8000709503C040E050E0BA01C695C695C370A6
:100E90008A019B01082B192B2A2B3B2BC901B80176
:100EA000C23049F058F4C13019F00E94960981C04F
:100EB0000E9484097EC00E94A8097BC00E94F70896
:100EC00078C0CF70112339F08C2F0E941D098D2F0F
:100ED0000E94C2056EC08D2F0E94C9058C2F0E94F2
:100EE0003E0967C0D23F21F128F4D03F41F0D13F05
:100EF000C1F043C0D33F19F1D43F79F03EC0112374
:100F000041F0053008F051C08C2F8F710E946309A9
:100F10004CC0063008F049C0F7CF8091FF0282FF35
:100F200018C0112339F08C2F8F710E941D093DC00C
:100F30001123C9F38C2F8F710E943E0936C01123F3
:100F400029F08C2F8F710E9408092FC00E9403097D
:100F50002CC0112349F0CF718C2F0E941D0963E032
:100F60008C2F0E943F0E21C081E00E945A0E023059
:100F7000E0F082E00E945A0E18C0112331F00023E5
:100F800091F28D2F0E94900410C0002399F2D93362
:100F900049F41FEF27EE33E0115020403040E1F7D5
:100FA00000C000008D2F0E943A0588EF8C0D843020
:100FB00020F40E941F200E942504DD20C9F00E9419
:100FC000AD0D80FD15C0F70112820E94A70D0E9491
:100FD0001D09C7010E9419080E94A70DDF91CF913A
:100FE0001F910F91FF90EF90DF90CF900C943E09EE
:100FF000DF91CF911F910F91FF90EF90DF90CF90F5
:1010000008950F931F93CF93DF93EC01688179814B
:101010008A810E945F0A8C010E94BA090E94AB0873
:10102000B801CE010E94D005DF91CF911F910F91A1
:101030000895CF93DF93EC01988189812B813C81C6
:10104000232B31F08F3F31F481E09F3F19F403C02F
:1010500081E001C080E080FD1DC0CE010E94A4039C
:10106000811110C00E94B10D8823A1F08A818823CC
:1010700089F08091FF0282FD0DC082E0DF91CF9167
:101080000C945A0ECE010E940108CE01DF91CF913F
:101090000C948503DF91CF91089580E090E00E9449
:1010A000532080E090E00E9469200E94D80D0E94A9
:1010B000FA0D0E9469160C943815809102019091E6
:1010C00003010E942B210C944D080E94C80D0C9422
:1010D0005D0892959F70963079F010F4925001C09F
:1010E0009A50923068F4803F69F018F4883E40F4DA
:1010F00009C0843F29F406C0883E20F0813F11F0EA
:1011000080E0089581E00895FC01808191810E9432
:10111000540A0E9469080895CF93DF9300D000D04D
:101120001F92CDB7DEB70F900F900F900F900F90DA
:10113000DF91CF910895CF93DF9300D000D000D0FE
:10114000CDB7DEB726960FB6F894DEBF0FBECDBF83
:10115000DF91CF910895089508950C94AC080C94F4
:10116000AD080E94AF086093180270931902809333
:101170001A0290931B020C944D080C94B1080F9323
:101180001F93009118021091190220911A023091B8
:101190001B02602B712B822B932B1F910F910C94B0
:1011A000B1080F931F93009118021091190220911A
:1011B0001A0230911B0260237123822393231F9113
:1011C0000F910C94B1080F931F9300911802109186
:1011D000190220911A0230911B0260277127822781
:1011E00093271F910F910C94B1080C94AC080E94A6
:1011F000F508609314027093150280931602909381
:1012000017020C944D0860E070E0CB010C94F708D5
:101210000F931F9341E050E060E070E08A019B0172
:1012200004C0000F111F221F331F8A95D2F7C90176
:10123000B8011F910F910C94F7080F931F9341E091
:1012400050E060E070E004C0440F551F661F771F38
:101250008A95D2F78091140290911502A0911602FE
:10126000B09117028A019B01082B192B2A2B3B2BCB
:10127000C901B8011F910F910C94F7080F931F93A8
:1012800041E050E060E070E004C0440F551F661F6D
:10129000771F8A95D2F7409550956095709580910B
:1012A000140290911502A0911602B09117028A01C2
:1012B0009B01082319232A233B23C901B8011F914D
:1012C0000F910C94F7080F931F9341E050E060E0FA
:1012D00070E004C0440F551F661F771F8A95D2F730
:1012E0008091140290911502A0911602B0911702FC
:1012F0008A019B01082719272A273B27C901B80122
:101300001F910F910C94F7080F931F9300911402F3
:10131000109115022091160230911702602B712B4B
:10132000822B932B1F910F910C94F7080F931F930F
:1013300000911402109115022091160230911702AB
:1013400060237123822393231F910F910C94F7083C
:101350000F931F9300911402109115022091160211
:101360003091170260277127822793271F910F91D1
:101370000C94F70808952FE0929F800D1124E82F18
:10138000E695E695E695877051E001C0550F8A9580
:10139000EAF785E0E89FF0011124E253FE4F20E0D8
:1013A00030E070E04081CB01022E02C09695879517
:1013B0000A94E2F78170819584278523842781939D
:1013C0002F5F3F4F2530310569F708952FE0929F39
:1013D000800D1124682F669566956695982F9770F5
:1013E00085E0689FB001112440E050E080E0FB01FF
:1013F000E40FF51FE253FE4F208130E0092E02C0BA
:10140000369527950A94E2F721703327042E01C000
:10141000220F0A94EAF7822B4F5F5F4F4530510548
:1014200031F70895BF92CF92DF92EF92FF920F9320
:101430001F93CF93DF938C01C0901402D0901502BC
:10144000E0901602F0901702809118029091190214
:10145000A0911A02B0911B02C82AD92AEA2AFB2AB3
:10146000CFE1D0E0D701C6010C2E04C0B695A795F8
:10147000979587950A94D2F780FD04C0219790F73D
:10148000B12C07C0BC2EB8018C2F0E945F110197B0
:10149000A9F38B2DDF91CF911F910F91FF90EF90CA
:1014A000DF90CF90BF900895CF93DF93EC010E941F
:1014B000120ABE010E945F11DF91CF9108951F9320
:1014C000CF93DF93EB019091CD01992321F0CB01D4
:1014D0000E94540A13C0882349F0CB010E94120ACB
:1014E000182F682FCE010E94BB0904C0CB010E94B7
:1014F000E609182FBE01812F0E945F11DF91CF9165
:101500001F9108951F93CF93DF93C0911C0216E0A3
:1015100080911D02C81799F0D0E01C9FF0011D9F1B
:10152000F00D1124E25EFD4F408151816281738193
:10153000848195810E949B082196C770E9CFDF9135
:10154000CF911F91089540914E0250914F026091AA
:1015500050027091510280915202909153020C946A
:101560009B08EF92FF920F931F93CF93DF9380918D
:10157000530282958F7009F065C0809150028823D4
:1015800009F460C080911C02F0901D0210914E027F
:1015900000914F02609151027091520291E01F3F01
:1015A00009F090E0C0910001D0910101292F96E04F
:1015B000E92E8F1509F446C06115710521F00F3F22
:1015C00021F030E003C031E001C0322F90E030FD67
:1015D00036C0E89EF001E99EF00D1124DF01A25E05
:1015E000BD4F11963C911197301329C03C91311396
:1015F00026C012963C911297311121C013964D913D
:101600005C911497461B570B4C175D07C0F48091F3
:1016100053028F70806180935302ED5DFD4F808196
:101620008F70806180838EE492E00E941908DF91C0
:10163000CF911F910F91FF90EF900C94820A019629
:101640008770B7CFDF91CF911F910F91FF90EF90EF
:1016500008959F92AF92BF92CF92DF92EF92FF9246
:101660000F931F93CF93DF93CDB7DEB761970FB67C
:10167000F894DEBF0FBECDBF8C0185E0F801DE011E
:101680001D9601900D928A95E1F7D8011296EC9083
:1016900090914E02E0914F022091510230915202FE
:1016A0002115310531F0EF3F31F481E09F3F19F40E
:1016B00003C081E001C080E0B82FB1709B2E80FD97
:1016C00047C1D8014C9111965C9111971396AD903A
:1016D000BC9014978EE4C82E82E0D82EF090500271
:1016E000B501621B730B2091000130910101FF20B5
:1016F00009F4D9C0809153026217730708F095C0AE
:10170000282F207F09F052C05E1313C0491311C067
:10171000FE2CE1100EC08F708061809353020E94F6
:10172000A30AC6010E94190880915302F80185831B
:101730004DC1AB2831F05F3F31F481E04F3F19F4E8
:1017400003C081E001C080E080FD03C081E08E2500
:1017500002C080E090E0F82FF170FF2E80FF1CC0E7
:1017600080911C0220911D0236E0821709F40BC102
:1017700090E0389FF001399FF00D1124E25EFD4F9B
:101780006181561306C06081461303C06281E61270
:1017900003C001968770E9CFFE2CEE2009F416C134
:1017A0008091530281608093530254C05E1306C03F
:1017B000491304C0E11002C0F80199C0C8010E9499
:1017C0008408882361F1EE2051F120915302822F89
:1017D00082958F7090E0029774F080914E02909104
:1017E0004F0298878F831986BB86AA862C87CE01E5
:1017F00007960E94190886E0F801AEE4B2E0019075
:101800000D928A95E1F70E94B10A0E94A30A0AC0CC
:101810005E1711F1C8010E94840881112CC0C80113
:101820000E941908FF24F394D1C0282F207F81F74C
:101830007A2DB98AA88A6E2D89890E948C088EE437
:1018400092E00E94190886E0D6011D928A95E9F778
:101850000E94A30AF12CBAC04913DCCFE110DACF01
:10186000F8018583C8010E94190886E0D6011D92FF
:101870008A95E9F7ABC0EE2091F220915302822FB6
:1018800082958F7090E002970CF4B5CF80914E0254
:1018900090914F029A8389831B82BD82AC822E83F2
:1018A000CE010196A6CF6217730708F044C0FE2C44
:1018B000EE2009F4B4CF5E1330C049132EC020913E
:1018C000530220FD21C0822F82958F70482F50E057
:1018D00041155105C9F0F80125834F30510541F0FC
:1018E0008F5F982F9295907F822F8F70892B8583A1
:1018F000C8010E94190886E0F801AEE4B2E0019048
:101900000D928A95E1F73CC086E0F801AEE4B2E0C2
:1019100001900D928A95E1F759C0C8010E94840890
:10192000811169CF80915302816080935302C80175
:101930000E9419084BC07A2DB98AA88A6E2D898910
:101940000E948C0886E0D6011D928A95E9F718C09E
:10195000EE2009F464CFC8010E948408F82E882381
:1019600009F45DCF86E0F801AEE4B2E001900D929B
:101970008A95E1F78EE492E00E948A040E94B10AFF
:101980000E94A30A23C04D875E878D859E850E9495
:10199000540A292F22952F70223028F49F7039F095
:1019A000811105C00BC0243028F49F7049F4805E7B
:1019B000883020F0C8010E9419089F2CF92C06C01D
:1019C000D80115969C91907F91F7F8CF8F2D619655
:1019D0000FB6F894DEBF0FBECDBFDF91CF911F9140
:1019E0000F91FF90EF90DF90CF90BF90AF909F90BE
:1019F00008951F93CF93DF93CDB7DEB72C970FB623
:101A0000F894DEBF0FBECDBF4F83588769877A87B2
:101A10008B879C87CE0107960E94290B8823D1F0E3
:101A20009F8188852A853B85232B31F08F3F31F4B8
:101A300081E09F3F19F403C081E001C080E080FD98
:101A400047C04F81588569857A858B859C850E9422
:101A50009B083EC086E0FE013796DE01119601909C
:101A60000D928A95E1F7FF81E8856A857B8561158E
:101A7000710531F0EF3F31F481E0FF3F19F403C00D
:101A800081E001C080E080FD23C020911D0230E094
:101A9000C90101968770992740911C0250E0841774
:101AA0009507F1F1F983EA837D836C8396E0929F39
:101AB000D001939FB00D1124A25EBD4FFE0131965F
:101AC00001900D929A95E1F780931D020E94820A7F
:101AD00016E080911C0290911D02891771F1189FE8
:101AE000C0011124825E9D4F0E94290B882329F199
:101AF000E0911C021E9FF0011124E25EFD4F408127
:101B0000518162817381848195810E949B088091BB
:101B10001C0290E001968770992780931C02D9CF10
:101B20000E94650810921D0210921C02EEE4F2E081
:101B300086E0DF011D928A95E9F72C960FB6F8949E
:101B4000DEBF0FBECDBFDF91CF911F910895809171
:101B500074028595859585950895809174028770A6
:101B6000089590917402977081E009F480E00895DF
:101B700080919702089590919702892B8093970204
:101B800008958095909197028923809397020895F4
:101B900010929702089590919602892B8093960255
:101BA00008958095909196028923809396020895D6
:101BB00010929602089580917502089508950C94EC
:101BC000DE0D0C94DF0D9091FF0292FD08C0909104
:101BD0007502981721F0809375020C94E10D089519
:101BE00080917502882329F01092750280E00C9490
:101BF000E10D0895CF93DF93E0910201F09103018D
:101C0000809197028083E0910201F091030190811D
:101C100080919602892B808380917502882381F0C0
:101C2000E0910201F09103019081892B80838091E2
:101C30000201909103010E947F2081110E94F00D0A
:101C4000C0910201D091030140E250E064E572E0EE
:101C5000CE010E94D329892B69F080E2FE01A4E520
:101C6000B2E001900D928A95E1F7CE01DF91CF911C
:101C70000C942B20DF91CF9108950C94DE0D909160
:101C8000FF0292FD10C098E0899F90011124262B3D
:101C9000209374020E941D09809174028595859598
:101CA00085950C943D0E0C941D091092740280E0F1
:101CB0000C943D0E209174028095822380937402CF
:101CC000982F977099F430E0482F082E000C550B90
:101CD0002417350759F09091FF0292FD07C08595B2
:101CE000859585950E943E090C94550E0895909116
:101CF000FF0292FB222720F9281769F080FB92F956
:101D00009093FF028091FE029091FF020E94C50E07
:101D100082E00C945A0E08958091FF0282FB88277E
:101D200080F991E089270C94770E81E00C94770E6E
:101D300080E00C94770E6FEF7FEF80E090E00C94E2
:101D4000122A80E090E00E94EE2921E0893E9E4F19
:101D500009F020E0822F089582E090E00C94E029C1
:101D600083E090E00C94E029CF9384E090E00E941F
:101D7000E029C82F82E290E00E94E0292C2F30E079
:101D8000A901582BCA01CF910895CF93C92F682F6D
:101D900084E090E00E94F4296C2F82E290E0CF91E1
:101DA0000C94F429AB01BC018FE090E00C94062A5E
:101DB000AB01BC0183E190E00C94062A60E070E086
:101DC000CB010C94D80E60E070E0CB010E94D20EE3
:101DD0000C94DE0E69EE7EEF80E090E00E94122A05
:101DE00060E082E090E00E94F42960E083E090E00F
:101DF0000E94F429109218021092190210921A02ED
:101E000010921B0260E084E090E00E94F42960E000
:101E100082E290E00E94F42960E085E090E00E9478
:101E2000F42960E086E090E00E94F4296FEF87E0FB
:101E300090E00E94F42940E050E0BA0188E090E090
:101E40000E94062A60E08DE090E00E94F42940E0C4
:101E500050E0BA0188E190E00E94062A60E087E144
:101E600090E00E94F42940E050E0BA018CE190E05B
:101E70000E94062A60E070E080E290E00E94122A50
:101E800040E050E0BA0188E190E00E94062A0C94FC
:101E9000E30E0C94EA0E682F8EE090E00C94F42987
:101EA0000E94E5216093AA027093AB028093AC027A
:101EB0009093AD026093A6027093A7028093A8024C
:101EC0009093A902089585B7806885BF85B780681B
:101ED00085BF089581E008950C946A0F08950C94CD
:101EE0006E0F0C946E0F0C94710F0C946E0F0C947B
:101EF000750F0C946E0F0E94630F8BE392E10E94AA
:101F000015200E94790F0C94770F0E946F0F0C948C
:101F10006E0F0E9455120C9420040E94D0210E9442
:101F20003A130E94890F0E94EB1B0C94730F5F926F
:101F30006F927F928F929F92AF92BF92CF92DF92D9
:101F4000EF92FF920F931F93CF93DF93CDB7DEB73E
:101F50002A970FB6F894DEBF0FBECDBF0E944F1375
:101F6000C82E81110E94500F38E9832E32E0932E43
:101F700000E010E0502E802F0E9479125C01F401E5
:101F8000619071904F016826792661147104B1F453
:101F90000F5F1F4F0730110569F78FEF89838A8321
:101FA0001B820E94D9218160782F9D838C83498177
:101FB0005A816B818D810E9440043AC08091AE02AB
:101FC00081FD0E948212D12CEE24E394F12CC301F6
:101FD0008E219F21892B29F10E946C0F8823A9F063
:101FE000DE825F82AE20BF2081E0AB2809F480E072
:101FF00088870E94D9218160782F9A8789874E81AE
:102000005F8168858A850E944004000F111FF801D6
:10201000E856FD4F80819181E826F926F182E08221
:1020200007C0D394EE0CFF1CFFE0DF12D0CFB0CF7F
:1020300081E0C11001C080E02A960FB6F894DEBF9F
:102040000FBECDBFDF91CF911F910F91FF90EF9009
:10205000DF90CF90BF90AF909F908F907F906F90C8
:102060005F9008950E94970F0E942F1C0E945615A2
:102070000C943504CF93DF930E946411EC01811519
:1020800021E5920708F045C0811530E5930708F077
:1020900094C0883E910528F5803E910508F0F8C06F
:1020A000883A910570F4853A910508F07CC081303A
:1020B000910509F475C008F4E8C0049708F0E8C079
:1020C000E4C08F3B910508F0E0C0C85AD0E0CC0FC7
:1020D000DD1FC35ADE4F0990D881C02DCE01946414
:1020E000D8C0811540E2940758F4811551E0950756
:1020F00008F0CEC08D3E910508F4C7C09065C9C0F8
:10210000C11580E4D80708F4C0C0DF70CE01906A22
:10211000C0C0811525E59207A8F4811534E5930721
:1021200008F095C0811543E5940708F07BC0811540
:1021300052E5950708F061C0D82FCC27CE01816FFA
:10214000906AA7C0C11589E5D807A0F4C11528E594
:10215000D20708F082C0C11536E5D30708F095C054
:102160008C2F0E94F8118F7190E0D82FCC27CE01D0
:1021700090628FC0C1154AE5D40708F474C0CE013F
:1021800090568115904208F080C08D2F8F710E946B
:10219000F811DD27D0628F71AE01582BCA0179C0CA
:1021A00081E090E076C0C55AD0E0C557DE4F888107
:1021B000C82FD0E0CE0190646CC074E096958795EE
:1021C0007A95E1F7282F23703C2F337081E090E05F
:1021D00002C0880F991F3A95E2F79C68AC01522B18
:1021E0009A019C2F9F709695969550E2959FE001DD
:1021F0001124C9018C2B9D2B4CC08370992721E0A1
:1022000030E002C0220F331F8A95E2F79C2F96958B
:10221000969580E2989FE0011124C22BD32BCE012A
:102220009C6837C08370992721E030E002C0220FFC
:10223000331F8A95E2F79C2F9695969540E2949FDE
:10224000E0011124C22BD32BCE019A6822C0D82FD3
:10225000CC27CE01846F906A1CC0DC2FCC27CE0126
:10226000806F906A16C08C2F8F700E94F81194E0D6
:10227000D695C7959A95E1F7CF70D0E0DC2FCC27A3
:10228000D0699E01282BC90104C080E090E001C004
:10229000CE01DF91CF91089529E6829FC0011124DC
:1022A000FC012FE0729FE00DF11D1124E60FF11DDE
:1022B000EE0FFF1FE852FF4F8591949108950E9401
:1022C0004C110E943A1008958238910569F1B0F4DA
:1022D0008133910509F46DC048F48932910509F400
:1022E00063C08A32910509F469C008958533910568
:1022F00009F455C089339105B9F00895833E9105DD
:1023000069F138F4803E9105B1F0823E910509F102
:102310000895863E9105A9F1873E9105B9F1843E65
:10232000910509F064C023C02091FE0220FD4FC03A
:1023300021FD4DC008958091FE0280FD44C0809132
:10234000FF0280FF44C08091FE0284FD42C083EE04
:102350004DC08091FE0282FF38C0F5CF8091FE0211
:1023600082FD33C08091FF0280FD31C0ECCF8091AF
:10237000FF0281FF32C08091FE0284FD2AC087EEF9
:1023800035C08091FE0283FF26C0F5CF8091FE020A
:1023900083FD21C08091FF0281FD1FC0ECCF8091A1
:1023A000FE0285FD1CC01DC08091FE0285FD19C086
:1023B00016C08091FE0286FD16C017C08091FE02F5
:1023C00086FD13C010C089E311C082EE0FC080EEFD
:1023D0000DC080E00BC086EE09C084EE07C089E224
:1023E00005C085E303C08AE201C081E390E008955F
:1023F0009091FE0292FF0DC0282F2871283019F409
:10240000877F846006C0282F2471243011F48B7FCD
:10241000886093FF0DC0282F2871283119F4877E1A
:10242000846106C0282F2471243111F48B7E8861C9
:102430002091FF0220FF0DC0382F3871383019F479
:10244000877F816006C0382F3171313011F48E7F63
:10245000886021FF0DC0282F2871283119F4877E4C
:10246000816106C0282F2171213111F48E7E88618F
:1024700094FD877E089580E008950C949B0E0E9441
:102480004F138FE39CE90197F1F700C000000E9411
:102490004F1380E00E94791280FF04C00E943D1219
:1024A0000C94262208950C943F120E94A10E8111D3
:1024B00002C00E94490F0E94AC0E8093AE020E949F
:1024C000B40E9093FF028093FE020E9453120E946A
:1024D000B00E682F70E080E090E00E94BD0860912F
:1024E00014027091150280911602909117020C94BB
:1024F000F508E82FF0E0EE0FFF1FE25FFC4F808150
:1025000091810895089580EA8A95F1F7089500C0B1
:1025100008950C94831208950C948B120C948C12D1
:102520000C948B120C949012F894E82FE295EF70B3
:10253000F0E031A1282F2F7081E090E001C0880FDA
:102540002A95EAF7982F9095932391A392A1892B2E
:1025500082A3789408950F931F93CF93DF93CDE9CF
:10256000D1E089918F3F11F00E94941281E0C43A2A
:10257000D807B9F7CEE8D1E00DE911E089918F3F96
:1025800011F00E9494120C171D07C1F7DF91CF9133
:102590001F910F910895BF92CF92DF92EF92FF9219
:1025A0000F931F93CF93DF938C01C62FD0E0CE0102
:1025B00083569E4F6C01FC0190819F3F09F450C0EF
:1025C000B62EF894E92FE295EF70F0E081A19F70AC
:1025D00021E030E001C0220F9A95EAF7822B81A317
:1025E00082A12095282322A378940E948712EEE8E6
:1025F000F1E04DE951E021E030E0E12CF12C619176
:102600006F3F89F0A62FA295AF70B0E090968C91A5
:1026100090E06F7002C0959587956A95E2F780FD0E
:1026200002C0C90102C080E090E0E82AF92A220F26
:10263000331F4E175F0719F7F60180818F3F11F0A6
:102640000E94941261E0E114F10409F460E08B2D22
:102650000E948912CC0FDD1FC00FD11FF982E882C2
:10266000DF91CF911F910F91FF90EF90DF90CF906E
:10267000BF9008950E94AB128EE0EEE0F3E0DF0120
:10268000982F1D929A95E9F7E0E0F3E0DF011D92A3
:102690008A95E9F787E00E949A130C949003FF92C1
:1026A0000F931F93CF93DF93CDB7DEB72E970FB65F
:1026B000F894DEBF0FBECDBF8E010F5F1F4F8EE0BF
:1026C000F80111928A95E9F7F12C6F2DC8010E944B
:1026D000CB12F394F7E0FF12F8CF4EE050E0B801D0
:1026E00080E093E00E94D329FF24F394009709F43B
:1026F000F12C892B41F08EE0F801A0E0B3E00190CD
:102700000D928A95E1F72F2D47E06EE073E080E0AF
:1027100093E00E949B130E9492038F2D2E960FB67A
:10272000F894DEBF0FBECDBFDF91CF911F910F9107
:10273000FF9008950895FF920F931F93CF93DF9317
:10274000F82E092F162FD72FC42F222349F081E00E
:102750008093B1020E94D9219093B0028093AF027E
:102760008091B1028823D9F08091AF029091B0029C
:102770000E94F121059798F0EF2DF02FA12FBD2F8A
:1027800080E090E04C2F50E08417950734F42191BD
:1027900031912D933D930196F7CF1092B102DF91C5
:1027A000CF911F910F91FF9008950E94F1230E94F5
:1027B0008D0F0C94FD230E9401240E9432100C9472
:1027C0001B240E9477210E94D8230E947B0F0E9425
:1027D000D5130E94DB130E94850FFBCF8091B802B6
:1027E00080FF06C06091090170E0660F771F26C068
:1027F00081FF04C06091090184E005C082FF07C029
:102800006091090188E0689FB001112417C0909180
:10281000B7029923D1F060910801961788F72091AB
:10282000090188E0289F90011124929FA001939FA5
:10283000500D112470E0CA010E944D2960387105C5
:1028400040F46115710519F406C068E070E0862F48
:1028500008958FE7089581E008958091B80280FF80
:1028600008C06091050170E075956795759567954D
:1028700021C081FF06C06091050170E075956795E4
:1028800019C082FF04C06091050170E010C09091F2
:10289000B602992399F0609104019617A0F78091F0
:1028A0000501899FC001112470E00E944D29603804
:1028B000710540F46115710519F406C061E070E01E
:1028C000862F08958FE7089581E008958D3E21F4C5
:1028D0000E94EE13819504C08E3E29F40E94EE13EF
:1028E0008093BC0208958F3E21F40E94EE138195DF
:1028F00004C0803F29F40E94EE138093BB02089528
:10290000893F19F40E942D1405C08A3F31F40E94BA
:102910002D1481958093BD0208958B3F21F40E9470
:102920002D14819504C08C3F29F40E942D148093AE
:10293000BE0208959FE0980F983078F421E030E0CF
:10294000A90102C0440F551F9A95E2F7CA01909160
:10295000BA02892B8093BA0208958D3F21F48091A9
:10296000B80281600BC08E3F21F48091B802826072
:1029700005C08F3F29F48091B80284608093B8022B
:1029800008958D3E39F49091BC0297FF35C01092A6
:10299000BC0259C08E3E29F49091BC021916BCF3BA
:1029A0002BC09091BB028F3E29F497FF25C0109257
:1029B000BB0249C0803F19F41916CCF31DC0909199
:1029C000BD02893F29F41916BCF41092BD023BC028
:1029D0008A3F19F497FF10C0F8CF8B3F39F49091DC
:1029E000BE0297FF09C01092BE022DC08C3F21F499
:1029F0009091BE021916BCF39FE0980F983080F4B6
:102A000021E030E0A90102C0440F551F9A95E2F77A
:102A1000CA0180959091BA0289238093BA0213C0AB
:102A20008D3F21F48091B8028E7F0BC08E3F21F440
:102A30008091B8028D7F05C08F3F29F48091B80244
:102A40008B7F8093B8028091BB02811106C0809178
:102A5000BC02811102C01092B7028091BD028111A7
:102A600006C08091BE02811102C01092B602089584
:102A70000E94D9212091BB02211104C02091BC02E7
:102A8000222321F09093B5028093B4022091BD02DD
:102A9000211104C02091BE02222321F09093B302A1
:102AA0008093B20289EB92E00C944520EF92FF9262
:102AB0000F931F93CF93DF9300D000D000D0CDB7FA
:102AC000DEB786E0E9EBF2E0DE01119601900D92AF
:102AD0008A95E1F7E090BB02F090BC020091BD0244
:102AE0001091BE021092BB021092BC021092BD0265
:102AF0001092BE02E11003C0FF2009F45DC0809176
:102B0000B4029091B5020E94F121AC019091B702FC
:102B1000992339F020910A0130E02417350758F045
:102B20004BC020910B018AE0289F900111242417AB
:102B3000350718F041C09F3F19F09F5F9093B7028F
:102B4000EE2061F00E94EE131E1414F09FEF01C0FE
:102B500091E0989F902D11249093BB02FF2061F08B
:102B60000E94EE131F1414F09FEF01C091E0989F94
:102B7000902D11249093BC023091BB023323E1F0DD
:102B80002091BC022223C1F045EB3403C001112483
:102B9000992319F09093BB0203C081E08093BB029C
:102BA00035EB2303C0011124992319F09093BC0243
:102BB00003C081E08093BC02011103C0112309F41A
:102BC0005DC08091B2029091B3020E94F121AC01EC
:102BD0009091B602992339F02091060130E0241734
:102BE000350758F04BC0209107018AE0289F9001DB
:102BF00011242417350718F041C09F3F19F09F5F3B
:102C00009093B602002361F00E942D14101614F068
:102C10009FEF01C091E0989F902D11249093BD02E9
:102C2000112361F00E942D14111614F09FEF01C0C2
:102C300091E0989F902D11249093BE023091BD0297
:102C40003323E1F02091BE022223C1F045EB34038F
:102C5000C0011124992319F09093BD0203C081E0B3
:102C60008093BD0235EB2303C0011124992319F091
:102C70009093BE0203C081E08093BE028091BB02AC
:102C800081110BC08091BC02811107C08091BD02EF
:102C9000811103C08091BE0281110E943815EB8220
:102CA000FC820D831E8386E0FE013196A9EBB2E023
:102CB00001900D928A95E1F726960FB6F894DEBF43
:102CC0000FBECDBFDF91CF911F910F91FF90EF907D
:102CD0000895E9EBF2E086E0DF011D928A95E9F7BD
:102CE0001092B7021092B6021092B8020895EF92B5
:102CF000FF920F931F93CF93DF938B01682F1111D6
:102D00000AC0442329F0E82FF0E0ED56FC4F64910F
:102D1000762F862F75C0212F30E0E82FF0E0442376
:102D200021F0ED56FC4FE491F0E046E0049FC00135
:102D30001124CFEFD0E0BE010E9439294BEA4603AF
:102D4000C001479F900D1124800F911D800F911D90
:102D5000982F990F890FAE01421B530B4E9FD00144
:102D60004F9FB00D5E9FB00D11249B2F189FA001A7
:102D70001124452F55278E01041B150B0E9FA00112
:102D80000F9F500D1E9F500D11247E01E81AF1086F
:102D9000E29E8001E39E100DF29E100D1124212F62
:102DA0003327C21BD30BCE9F9001CF9F300DDE9FE8
:102DB000300D112462307105A9F048F461157105D8
:102DC00069F061307105C9F48B2F752F0DC0643027
:102DD000710581F058F06630710579F47E2F8B2FE4
:102DE000932F0DC0832F7B2F9E2F09C08E2F7B2FFB
:102DF000952F05C08E2F732F02C07E2F852F692F30
:102E0000DF91CF911F910F91FF90EF90089541E0D6
:102E10000E947716089508950E9407170895CF938A
:102E2000DF93762FE901682F842F0E940C17798396
:102E300068838A83DF91CF91089580911C03282FA6
:102E4000269530E02115310519F48170826005C0A6
:102E50002532310524F08170886480931C03089525
:102E600088E090E00C94E829CF92DF92EF92FF92F5
:102E70006B017C010E941D17B701A60188E090E05C
:102E8000FF90EF90DF90CF900C94062AECE1F3E0F6
:102E900083E0808311828FEF828383831482608139
:102EA0007181828193810C94341780911C0380FF7F
:102EB00002C08695089580E0089590912003933094
:102EC00018F49F5F90932003882351F060911C03B6
:102ED00070911D0380911E0390911F030C94341771
:102EE000089581E00C945D1790912003992319F0C7
:102EF000915090932003882351F060911C037091AE
:102F00001D0380911E0390911F030C9434170895A4
:102F100081E00C94741770E00C94AC1D609110016A
:102F200080911C0380FF0AC080910F0123E0829FE3
:102F3000C00111248F5D9C4F0C948B17809111015F
:102F400090911201891780F7E82FF0E09F01220F7E
:102F5000331FE20FF31FEF5DFC4F118210821282CC
:102F60008F5FF0CF90911C0390FF16C090911101DC
:102F700020911201921770F4E92FF0E0DF01AA0FFF
:102F8000BB1FEA0FFB1FEF5DFC4F81836083428311
:102F90009F5FF0CF0C948E170895CF93DF9300D0EE
:102FA0001F92CDB7DEB790911C0390FF0AC09E011F
:102FB0002F5F3F4F0E940F174B8169818A810E94CA
:102FC000B2170F900F900F90DF91CF910895CF938C
:102FD000DF93EC01EC81F0E0E257FD4F4491ECE12E
:102FE000F3E0628181810E94CD178C818F5F8C8399
:102FF000DF91CF910895CF93DF93EC01ECE1F3E003
:10300000438162818C810E94CD178C818F5F8C837C
:10301000DF91CF9108950F931F93CF93DF9300D04B
:103020001F92CDB7DEB78C018091BF0281110AC01B
:103030009E012F5F3F4F4FEF6FEF0E940F178A8166
:103040008093BF02F8018481813051F028F08230F2
:1030500061F44091BF020AC08091BF0240E007C006
:103060006091BF0240E080E003C040E080E060E0AB
:103070000E94B217F801848190E0019663E070E04D
:103080000E944D2984830F900F900F90DF91CF9174
:103090001F910F910895AF92BF92CF92DF92EF925E
:1030A000FF920F931F93CF93DF9300D01F92CDB762
:1030B000DEB7182FF62E042FE22E90911C0390FFFE
:1030C0006DC0E92FE695AE2FB0E0AC55BE4F8C91A8
:1030D0008093CB029E7F923061F49E012F5F3F4F21
:1030E000812F0E940F174B8169818A810E94B2173C
:1030F00043C0823019F400911F033EC0863019F49A
:1031000010911D0339C08930D9F38931A9F5E951EE
:103110008E2F8170D82EE695F0E0E257FC4FA590F7
:10312000B490C12CBB2460911301C61618F52C2D48
:1031300030E0A29EC001A39E900DB29E900D11247E
:1031400070E00E943929812FD11002C0860F01C082
:10315000861B90911101290F311DA901440F551FA4
:10316000240F351F2F5D3C4F402F6F2D0E940F17EE
:10317000C394D9CF0E948E1710931D03F0921E03A3
:1031800000931F03EE2051F060911C0370911D030A
:1031900080911E0390911F030E9434170F900F908F
:1031A0000F90DF91CF911F910F91FF90EF90DF90E3
:1031B000CF90BF90AF900895ECE1F3E09181282F7C
:1031C0004381628188E0890F0C944B1881E00C9454
:1031D000DC18ECE1F3E09181282F4381628188EFD4
:1031E000890F0C944B1881E00C94E918ECE1F3E0A2
:1031F000628128E0620F08F46FEF282F43818181FC
:103200000C944B1881E00C94F618ECE1F3E0628129
:1032100028E0621B08F460E0282F438181810C9430
:103220004B1881E00C940519ECE1F3E0438128E0B0
:10323000420F08F44FEF282F628181810C944B18C4
:1032400081E00C941419ECE1F3E0438128E0421B87
:1032500008F440E0282F628181810C944B1881E0B2
:103260000C94231920E00C944B18FF920F931F939A
:10327000CF93DF93EC01F12C0FEF10E0609113017D
:10328000F616F0F4809111012F2D30E0280F311D3A
:10329000C901880F991F280F391F2F5D3C4F70E01F
:1032A000C8010E944D29962F8C8140911F03609187
:1032B0001E03F99E800D11240E940F17F394DECF98
:1032C0000E948E179A818C8190FF02C08F5F01C08F
:1032D00081508C83DF91CF911F910F91FF900895C2
:1032E000AF92BF92CF92DF92EF92FF920F931F9314
:1032F000CF93DF93FC01828180FF02C00FEF01C0FA
:1033000001E010E049E2A42E80911301181708F0A3
:1033100043C080911101C12ED12CE601C80FD11DEF
:10332000CE01880F991FC80FD91FCF5DDC4F1982BE
:1033300018821A8234E0E32EF12CB12C8091C10264
:103340008B0D8A322CF06A2D0E942B29892F05C003
:1033500087FF03C090911301890F082E000C990B71
:10336000C816D90691F480911F038E9DA0018F9DF0
:10337000500D112455954795559547959E0160919F
:103380001E0380911D030E940F17B00EF1E0EF1A8B
:10339000F108A1F61F5FB8CF0E948E178091C1027D
:1033A000013031F4811102C080911301815007C0B6
:1033B00090E001966091130170E00E944D29809386
:1033C000C102DF91CF911F910F91FF90EF90DF909D
:1033D000CF90BF90AF900895CF93809111019091BD
:1033E0001201891770F4E82FF0E09F01220F331FBC
:1033F000E20FF31FEF5DFC4F1182108212828F5F8C
:10340000F0CFC0E060911301C617C0F5EC2FF0E0DB
:1034100070E0CF010E944D2920911101820F20916F
:10342000C002022E000C330B90E0E217F307CCF041
:1034300020910E01022E000C330B2E173F078CF04B
:103440009C01220F331F820F931F9C012F5D3C4F65
:1034500040911F0360911E0380911D030E940F176E
:103460000BC0FC01EE0FFF1F8E0F9F1FFC01EF5DD5
:10347000FC4F118210821282CF5FC4CF0E948E1740
:1034800020910D018091C002820F8093C002909123
:103490000E01920F90930E0119165CF4082E000C89
:1034A000990B4091130150E0415051098417950741
:1034B0001CF0219520930D01CF9108958F929F923A
:1034C000AF92BF92CF92DF92EF92FF920F931F9332
:1034D000CF93DF938C01FC014481C42FD0E09E0187
:1034E000DE010E9491299B01AC010E94A7296B017A
:1034F0007C01E0E2F0E0EC1BFD0BA5E5B0E09B01F8
:10350000AC010E94A7294B015C019F01DF010E94D1
:1035100089299B01AC010E94B2299B01AC012C0DB1
:103520003D1D4E1D5F1DC501B4010E946129C22FC2
:10353000D22F2A3228F4F3E02F9F900111240DC0DE
:1035400025E530E02C1B3109C901880F991F280F90
:10355000391F37FF02C02F5F3F4F35952795C22F88
:10356000C095F12C85E5E82EED1A80911301F8162F
:10357000C8F4F1FC02C08E2D01C08D2F9091110175
:103580002F2D30E0290F311DA901440F551F240FA5
:10359000351F2F5D3C4F4C2F60911E030E940F176B
:1035A000F394E3CF0E948E17F8018481811102C049
:1035B00091E003C0803219F49FEF90930C01909139
:1035C0000C01890FF8018483DF91CF911F910F9136
:1035D000FF90EF90DF90CF90BF90AF909F908F9033
:1035E00008950F931F93CF93DF93EC0100E010E059
:1035F00080911301282F30E00217130724F59091D2
:1036000011019801290F311DA901440F551F240FE5
:10361000351F2F5D3C4F869590E04C8108171907A8
:103620001CF4442331F002C0411103C040911F0338
:1036300001C040E060911E0380911D030E940F179E
:103640000F5F1F4FD5CF0E948E178C8190E001969F
:10365000817099278C83DF91CF911F910F910895ED
:10366000ECE1F3E080818E7F8083608171818281D3
:1036700093810E9434171092CC022FEF80E792E0E2
:10368000215080409040E1F700C000000C948E175C
:10369000ECE1F3E080818E7F80831092CC022FEFEB
:1036A00080E792E0215080409040E1F700C00000A8
:1036B0000C948E171092CC028091C90281110AC01D
:1036C00081E08093C90280911C0381708093C802BD
:1036D0000C94481B089560911C03669570E04BE0C4
:1036E00050E084E191E00E94C629892B19F481E021
:1036F0008093CC020E94D9219093C3028093C2028E
:10370000089590911C0390FF35C09170811102C003
:10371000926006C0853210F0986402C0880F982B22
:1037200090931C03662351F060911C0370911D035C
:1037300080911E0390911F030E94341760911C0317
:10374000669570E04BE050E084E191E00E94C6296C
:10375000892B19F01092CC0202C00E946B1B81E0F1
:103760008093C50240911F0360911E0380911D0349
:103770000C9432190895682F90911C03969581E05E
:10378000890F853208F081E00C94811B81E00C9454
:10379000BB1B682F90911C0396958FEF890F09F43E
:1037A00084E20C94811B81E00C94C91B61E00C94B1
:1037B000811BECE1F3E080818160808386950C942D
:1037C000D61B80911C0380FD0C94301B0C94D91BDC
:1037D00060E00C94811B8091CA0281112EC00E946E
:1037E000A10E811104C00E94490F0E9446170E9439
:1037F000301760931C0370931D0380931E039093F6
:103800001F036E7F61F40E9446170E943017609379
:103810001C0370931D0380931E0390931F030E944B
:103820001D171092CC0280911C0380FF03C0869567
:103830000E94E81B81E08093CA020895ECE1F3E066
:1038400080818160808386950C94E81B1092C90268
:103850008091C80281110E941E1C0C946B1B0F9357
:103860001F93CF93DF938091CC02882309F485C006
:103870008091CB02E0911C03E695E81BE093C40223
:10388000823049F4F0E0E657FD4FE491CE2FD0E0CE
:1038900007EE17E149C0863049F4F0E0E957FD4FE3
:1038A000E491CE2FD0E00BEF17E13EC0893051F408
:1038B000E695F0E0EC57FD4FE491CE2FD0E005E324
:1038C00019E132C08F3051F4E695F0E0EF57FD4F2B
:1038D000E491CE2FD0E000E719E126C0853149F40C
:1038E000F0E0E258FD4FE491CE2FD0E00CEE19E16C
:1038F0001BC0883181F0833239F4ECE7F2E0C591E6
:10390000D4910BE018E110C0843251F4C4EFD1E03F
:1039100001EF1AE109C0C8E2D0E00EE51AE104C0E7
:10392000C0EDD7E00BE017E18091C502882361F07C
:103930001092C5020E94D9219093C3028093C202C3
:103940001092C7021092C6020E94D921E091C202D1
:10395000F091C3028E1B9F0B8F3F9F4770F4EC0FBB
:10396000FD1FF093C302E093C20282EC92E0F801E3
:10397000DF91CF911F910F910994DF91CF911F910A
:103980000F910895882311F0FA0101C0FB010994F9
:10399000CF93DF93C82FD62F0E9455178C1740F076
:1039A0000E9455178D1720F4DF91CF910C94C61B00
:1039B0008C2FDF91CF910C94D61B1F93CF93DF9365
:1039C000FB0112811111C3C0EC010E94B80D82727B
:1039D000CD3CFCE5DF0709F49AC0A8F5C73CECE54F
:1039E000DE0709F476C0A8F4C43C9CE5D90709F4C5
:1039F0005FC028F4C33CDC4509F457C054C0C53C43
:103A00009CE5D90709F459C0C63CDC4509F45CC003
:103A10004AC0CA3CFCE5DF0709F46AC050F4C83C60
:103A2000ECE5DE0709F45AC0C93CDC4509F45BC08B
:103A30003AC0CB3C9CE5D90709F45FC0CC3CDC45DF
:103A400009F460C030C0C23DFCE5DF0709F46FC077
:103A500088F4CF3C9CE5D90709F460C008F45CC049
:103A6000C03DFCE5DF0709F45CC0C13DDC4509F45D
:103A70005BC019C0C53D9CE5D90709F460C050F48E
:103A8000C33DFCE5DF0709F455C0C43DDC4509F43E
:103A900054C009C0C63D9CE5D90709F455C0CE35D0
:103AA000DD4509F454C011E052C00E94E11B4FC033
:103AB00043ED5BE166EC7BE104C046EC5BE163ED6A
:103AC0007BE10E94C21C43C043EF58E166EE78E1FF
:103AD000F8CF46EE58E163EF78E1F3CF41E159E1E9
:103AE00062E079E1EECF42E059E161E179E1E9CFCD
:103AF0004FE259E160E279E1E4CF40E259E16FE25F
:103B000079E1DFCF48E857E161E777E1DACF41E7D4
:103B100057E168E877E1D5CF81E017C065E082E042
:103B200010C068E086E00DC06EE089E00AC064E184
:103B30008FE007C067E185E104C088E106C062E26A
:103B400089E10E94C81C03C083E20E94D61B812F1A
:103B5000DF91CF911F910895209A25B12E7F35B125
:103B600031604FB7F894FC01CB01880F991F680FA3
:103B7000791F6E0F7F1FE617F70789F0819198E094
:103B800035B9000000C087FF25B9880F000000C0CC
:103B900000C000C025B900C09A9591F7ECCF4FBF87
:103BA0008FE594E00197F1F700C000000895CF93EE
:103BB000DF93EC01FB018281882309F43CC1C4300E
:103BC000FDE5DF0760F4CB3F9CE5D90788F49E0153
:103BD00022503C452431310508F02EC109C0C236BF
:103BE000EDE5DE0729F0C63AFDE5DF0709F024C15F
:103BF0000E94B40E9093FF028093FE02C1318CE5C7
:103C0000D80709F4C6C008F042C0C930ECE5DE07A9
:103C100009F49BC000F5C5308CE5D80709F485C0D0
:103C200078F4C330ECE5DE0709F478C008F07AC018
:103C3000C230DC4509F0F5C08091FE028160EFC022
:103C4000C7309CE5D90709F478C008F07AC08091A4
:103C5000FE028061E4C0CD30FCE5DF0709F487C0D7
:103C600058F4CB309CE5D90709F479C008F07BC043
:103C70008091FE0288606FC0CF30FCE5DF0709F459
:103C800080C008F082C08091FE02877FC8C0CE3F0E
:103C90009CE5D90709F471C000F5C531FCE5DF07E3
:103CA00009F485C068F4C3319CE5D90709F475C0EF
:103CB00008F095C00E9465088091FE028F77AFC022
:103CC000CC3FFCE5DF07A9F108F054C0CB3FDC4551
:103CD00009F0A7C08091FF0240C0C230EDE5DE07C9
:103CE00009F489C058F4C1158DE5D80709F45AC004
:103CF00008F069C08091FF0282602FC0C236EDE5F6
:103D0000DE0709F47CC0C63AFDE5DF0709F481C08F
:103D1000C330DD4509F085C080E06EC08091FE02B1
:103D200082607DC08091FE0216C08091FE02886094
:103D300076C08091FF0282604FC08091FE02806257
:103D40006EC08091FE0280646AC00E946508809106
:103D5000FE02806864C0846062C081603DC0809162
:103D6000FE028E7F5CC08091FE028D7F58C08091E4
:103D7000FE0216C08091FF0218C08091FF028D7F65
:103D80002BC08091FE028F7E4AC08091FE028F7D03
:103D900046C08091FE028F7B42C08091FE02877FE9
:103DA0008B7F3DC08091FF028D7F8E7F15C08091FB
:103DB000FE0282FB222720F991E0922790FB82F9F4
:103DC00090FB83F92CC08091FF02982F9095917001
:103DD0008E7F892B90FB81F98093FF0222C00E9485
:103DE00065088091FE0287FB222720F991E0922747
:103DF00090FB87F914C081E00E944B0F12C08091A4
:103E0000FE0284FB222720F991E0922790FB84F99F
:103E100006C08091FE02982F909590FB80F98093C8
:103E2000FE028091FE029091FF020E94C50E0E9448
:103E3000650880E001C081E0DF91CF910895CF93C4
:103E4000DF9386319C4541F5EB010E94B80D982F18
:103E50008A812091020130910301882379F09A7AB6
:103E600081E009F480E08093CD02911102C069E203
:103E700001C065E3C9010E9415210AC08091CD02ED
:103E8000811102C069E201C065E3C9010E942021DD
:103E90000E94FA0D80E001C081E0DF91CF9108958A
:103EA0000F931F93CF93DF93C42FD22FFC018281F6
:103EB0008823C9F04093D0020E94D9219093CF0269
:103EC0008093CE0280E28C0F883008F057C0C77014
:103ED00081E001C0880FCA95EAF7DF91CF911F9169
:103EE0000F910C94C2058091D002481330C080918C
:103EF000CE029091CF020E94F121883C910538F5C5
:103F000010E21D0FCD17B9F080E28C0F883040F41D
:103F1000C77081E001C0880FCA95EAF70E94C90501
:103F2000183028F581E09D2F977001C0880F9A9571
:103F3000EAF70E94C205802F0E94B9051830F0F4FC
:103F4000D77081E001C0880FDA95EAF70AC080E2F5
:103F50008C0F883098F4C77081E001C0880FCA9533
:103F6000EAF7DF91CF911F910F910C94C905802F33
:103F7000DF91CF911F910F910C94B905DF91CF91F3
:103F80001F910F9108950F939C01CB01243F4CE5A5
:103F9000340731F188F4293DFCE53F07D9F02A3D8B
:103FA0004CE5340779F1283D3C45A9F506E221EEC0
:103FB00041EE68ED7CE52BC0263FFCE53F07E1F0D4
:103FC000A8F0273F3C4539F507E225EE46EE67EFBE
:103FD0007CE51DC007E225EE45EE69ED7CE517C0E6
:103FE00006E221EE40EE64EF7CE511C007E225EE2B
:103FF00044EE65EF7CE50BC006E221EE42EE66EF93
:104000007CE505C008E221E045EE6AED7CE50E9412
:10401000501F80E008C0FC018281882319F01092B3
:10402000D00201C081E00F9108959093CB0180935D
:10403000CA0108959093D6028093D5020895E09125
:10404000D502F091D602309721F00190F081E02D59
:10405000099480E00895E091D502F091D60230975E
:1040600099F020912B01222359F02091FE0227FF85
:1040700007C0DC012C9111962C93119726E02C930C
:104080000280F381E02D09940895E091D502F0912A
:10409000D602309739F022E0DC012C930480F581C0
:1040A000E02D099408952091D3023091D40228176D
:1040B000390771F09093D4028093D302E091D50236
:1040C000F091D602309721F00680F781E02D099417
:1040D00008952091D1023091D2022817390771F04A
:1040E0009093D2028093D102E091D502F091D60252
:1040F000309721F00084F185E02D09940895FC01AA
:10410000329680912B01882331F08091FE0287FF47
:1041100002C09EE101C096E080E0915028F021911C
:104120002223D9F38F5FF9CF0895662351F12091AF
:104130002B012223E9F02091FE0227FF19C0462F10
:104140004695469546954E31E0F4677021E030E0A3
:1041500002C0220F331F6A95E2F7FC01E40FF11D44
:10416000828190E02823392381E0232B69F409C060
:10417000FC01329608962191621729F0E817F90799
:10418000D1F780E0089581E008959C01FC0132960A
:104190009FEF80E04191461789F09F3F19F441114C
:1041A00001C0982F8F5F8630A9F79F3F39F0F90142
:1041B000E90FF11D97FDFA956283089508959C011A
:1041C0002A5F3F4FFC014281461301C012820196D3
:1041D00082179307B9F70895262F269526952695D9
:1041E0002E3168F4FC01E20FF11D677021E030E030
:1041F00001C0220F6A95EAF78281282B2283089555
:10420000262F2695269526952E3170F4FC01E20F77
:10421000F11D677021E030E001C0220F6A95EAF7D6
:104220002095828128232283089520912B01222327
:1042300029F02091FE0227FD0C94EC200C94C5205F
:1042400020912B01222329F02091FE0227FD0C94BE
:1042500000210C94DF2020912B01FC0132962223B7
:1042600031F08091FE0287FF02C08EE101C086E03E
:10427000DF011D928A95E9F7089508950C943D2178
:1042800083E08093D7020C943E21811102C081E02B
:1042900001C082E08093D7020C943E210C9445210A
:1042A00081E08093D7020C943E210C945021089514
:1042B0000C9457210C9458210C9457210C9457219D
:1042C0000C945721CF930E945E210E944F130E94AD
:1042D0005C21C0E08C2F0E947912892B29F4CF5FDA
:1042E000C730C1F780E001C081E0CF910895089503
:1042F0001F920F920FB60F9211248F939F93AF933B
:10430000BF938091D802811113C080919C0390913A
:104310009D03A0919E03B0919F034196A11DB11DE5
:1043200080939C0390939D03A0939E03B0939F035F
:10433000BF91AF919F918F910F900FBE0F901F90E3
:1043400018958091A403843031F10E94FD031092EE
:10435000D80220E488E190E00FB6F894A895809305
:1043600060000FBE2093600083B7817F846083BFAD
:1043700083B7816083BF7894889583B78E7F83BF2E
:104380000FB6F894A89580916000886180936000D2
:10439000109260000FBE08950E9465080C940304FB
:1043A00082E084BD93E095BD9AEF97BD80936E0047
:1043B00008952FB7F89480919C0390919D03A0914C
:1043C0009E03B0919F032FBF08952FB7F89460917B
:1043D0009C0370919D0380919E0390919F032FBF3A
:1043E00008959C014FB7F89480919C0390919D0390
:1043F000A0919E03B0919F034FBF821B930B089522
:1044000078941F920F920FB60F9211248F939F935F
:10441000AF93BF9380919C0390919D03A0919E03C5
:10442000B0919F030196A11DB11D80939C039093B1
:104430009D03A0939E03B0939F03BF91AF919F9163
:104440008F910F900FBE0F901F90189581E0809371
:10445000E00080E28093D8001092C9008FE19EE4D2
:104460000197F1F700C0000087E090EBDC0180933A
:10447000AD039093AE03A093AF03B093B0039CE061
:1044800088E10FB6F894A895809360000FBE9093D2
:104490006000FFCF8091FC020895089522E02093F0
:1044A000E9002FEF3091E800215035FD06C035EDD1
:1044B0003A95F1F700002111F5CF2091E80025FF92
:1044C0000BC040E050E066E070E00E948D248091D7
:1044D000E8008E778093E8000895CF93DF932091D2
:1044E0002B01222339F02091FE0227FF03C060E256
:1044F00022E002C068E021E02093E9002FEF309134
:10450000E800215035FD06C035ED3A95F1F7000081
:104510002111F5CF2091E80025FF1DC0EC0180910D
:104520002B01811105C040E050E068E070E003C05D
:1045300070E040E050E0CE010E948D248091E800C0
:104540008E778093E80080E2FE01ACEDB2E001904E
:104550000D928A95E1F7DF91CF9108958093D9026A
:104560007093DB026093DA028091A403843001F53A
:1045700082E08093E9008FEF9091E800815095FDF3
:1045800006C095ED9A95F1F700008111F5CF809165
:10459000E80085FF0DC040E050E063E070E089ED89
:1045A00092E00E948D248091E8008E778093E8004D
:1045B0000895BC0184E00C94AE22BC0183E00C940D
:1045C000AE228091A303811109C00E941E260E9481
:1045D0007B268091E20084608093E200089510922F
:1045E000A30308950C9455216091A00381E061110B
:1045F00001C080E00C9440219091A40381E09430AC
:1046000009F080E06091A0030C94452142E061EC48
:1046100081E00E94972542E261EC82E00E949725AA
:104620009091A40381E0943009F080E06091A003B0
:104630000C944E218091A603833009F461C030F4BC
:10464000813071F0823009F49AC008958A3009F4FB
:1046500086C08B3009F46CC0893009F0A8C020C036
:104660008091A503813A09F0A2C08091E800877F7C
:104670008093E8008091A9039091AA03892B21F4EB
:1046800060E28CED92E003C060E080E090E070E0DA
:104690000E94D8248091E8008B778093E8000895E9
:1046A0008091A503813209F082C08091A903909185
:1046B000AA03029708F07BC08091E800877F80936F
:1046C000E8008091E80082FD05C08091A40381117B
:1046D000F8CF6DC02091F3008091F20090E0922B12
:1046E000029731F48091F100813011F0863021F48D
:1046F0008091F1008093FC028091E8008B7753C099
:104700008091A503813A09F052C08091A90390914C
:10471000AA03892B09F04BC08091E800877F809322
:10472000E8008091E80080FFFCCF80912B0136C02B
:104730008091A5038132D9F58091A9039091AA03B4
:10474000892BA9F58091E800877F8093E8000E947B
:10475000CC258091A70380932B010C946508809150
:10476000A503813221F58091E800877F8093E800DE
:104770000E94CC258091A8038093FD02089580912A
:10478000A503813AA1F48091E800877F8093E80037
:104790008091E80080FFFCCF8091FD028093F100C2
:1047A0008091E8008E778093E8000C94CC250895E2
:1047B00084B7877F84BF0FB6F894A8958091600076
:1047C000886180936000109260000FBE90E080E8E6
:1047D0000FB6F89480936100909361000FBE0C9423
:1047E00050210E941E260E947B26E2EEF0E080818E
:1047F0008460808378940C9410298FE191E00C946C
:104800001A208091A4038530A9F48091A4038530F7
:1048100079F40E94A1218091A2038823B1F30E9420
:104820006221882391F30E9477240E946508EDCFCE
:104830000C94CC21089508950C941E24292F33271D
:1048400023303105C9F060F42130310581F0223088
:10485000310509F044C08BE390E025EC34E043C01F
:1048600021323105E1F02232310549F138C082E1CF
:1048700090E020E035E037C099278130910549F07C
:1048800028F0029761F5E3E9F4E005C0E1ECF4E01B
:1048900002C0E5EAF4E0849190E09F0124C0611534
:1048A000710541F061307105D1F489E090E020EFAD
:1048B00034E019C089E090E027ED34E014C06115C0
:1048C000710541F06130710551F486EB90E022E111
:1048D00035E009C080E490E028EC35E004C080E0D9
:1048E00090E020E030E0FA0131832083089580E1F8
:1048F00089BD82E189BD09B400FEFDCF8091D80059
:104900008F7D8093D8008091E00082608093E000EA
:104910008091E00081FDFCCF0895CF92DF92EF926D
:10492000FF920F931F93CF93DF93EC018B017A01DA
:104930000E94EB25811133C0E114F10439F0F70135
:1049400080819181081B190BC80FD91FC12CD12C54
:104950000115110519F18091E80085FD16C08091BF
:10496000E8008E778093E800E114F10449F0F70144
:1049700080819181C80ED91ED182C08285E00FC08E
:104980000E94EB25882321F30AC089918093F100CE
:1049900001501109FFEFCF1ADF0ADACF80E0DF9173
:1049A000CF911F910F91FF90EF90DF90CF900895DE
:1049B0002091AB033091AC032617370748F06115FF
:1049C000710539F42091E8002E772093E80001C0AA
:1049D000B901FC0120E06115710579F18091A40312
:1049E0008823F1F18530F1F18091E80083FD3CC02E
:1049F0008091E80082FD2EC08091E80080FFEBCF1F
:104A00002091F3008091F20090E0922B61157105E6
:104A100051F08830910538F421912093F1006150D4
:104A200071090196F3CF21E0089709F020E0809109
:104A3000E8008E778093E800CECF2111CFCF0AC057
:104A40008091A403882361F0853061F08091E800B3
:104A500083FD0AC08091E80082FFF2CF80E00895D4
:104A600082E0089583E0089581E008952091AB03EA
:104A70003091AC032617370748F06115710539F4FA
:104A80002091E8002E772093E80001C0B901FC01D5
:104A900020E06115710591F18091A403882309F448
:104AA00040C0853009F43FC08091E80083FD3DC0DF
:104AB0008091E80082FD2FC08091E80080FFE9CF5F
:104AC0002091F3008091F20090E0922B6115710526
:104AD00059F08830910540F424912093F1003196EB
:104AE000615071090196F2CF21E0089709F020E0AA
:104AF0008091E8008E778093E800CBCF2111CCCF56
:104B00000AC08091A403882361F0853061F0809110
:104B1000E80083FD0AC08091E80082FFF2CF80E0C8
:104B2000089582E0089583E0089581E00895982F24
:104B3000973068F59093E900981739F07091EC0080
:104B40002091ED005091F00003C0242F762F50E00B
:104B500021FD02C09F5FECCF3091EB003E7F309390
:104B6000EB003091ED003D7F3093ED003091EB0094
:104B700031603093EB007093EC002093ED00509384
:104B8000F0002091EE0027FDE5CF80E008958F70C2
:104B90008093E90081E008958091A50387FF11C00B
:104BA0008091E80082FD05C08091A4038111F8CFB7
:104BB00011C08091E8008B770BC08091A4038823FB
:104BC00049F08091E80080FFF8CF8091E8008E776F
:104BD0008093E80008952091E4003091E50095E687
:104BE0004091EC00842F817040FF23C08091E80049
:104BF00080FD1DC08091A403882399F0853099F031
:104C00008091EB0085FD11C04091E4005091E500DA
:104C10002417350729F3915011F09A01E1CF84E070
:104C2000089582E0089583E0089581E0089580E08A
:104C300008954091E80042FFDDCF08950E948C2640
:104C40000E949426E0EEF0E0808181608083E8EDB0
:104C5000F0E080818F77808319BCA7EDB0E08C9164
:104C60008E7F8C9380818F7E80831092A303089522
:104C70000F931F93CF93DF930E948C260E9494265C
:104C8000C8EDD0E088818F778883888180688883A9
:104C900088818F7D888319BC1092A4031092A00391
:104CA0001092A2031092A10300EE10E0F80180819F
:104CB0008B7F808388818160888342E060E080E030
:104CC0000E949725E1EEF0E080818E7F8083E2EE06
:104CD000F0E0808181608083808188608083F8013A
:104CE00080818E7F8083888180618883DF91CF91EE
:104CF0001F910F910895E8EDF0E080818F7E808311
:104D0000E7EDF0E080818160808384E082BF81E014
:104D10008093A3030C943826E8EDF0E080818E7F29
:104D200080831092E20008951092DA001092E10060
:104D300008951F920F920FB60F9211242F933F9355
:104D40004F935F936F937F938F939F93AF93BF9393
:104D5000EF93FF938091E10082FF0BC08091E2000E
:104D600082FF07C08091E1008B7F8093E1000E9469
:104D70000F298091DA0080FF1FC08091D80080FF4A
:104D80001BC08091DA008E7F8093DA008091D90079
:104D900080FF0DC080E189BD82E189BD09B400FEBC
:104DA000FDCF81E08093A4030E94E12205C019BCDD
:104DB0001092A4030E94EF228091E10080FF19C0AD
:104DC0008091E20080FF15C08091E2008E7F809389
:104DD000E2008091E20080618093E2008091D8003F
:104DE00080628093D80019BC85E08093A4030E9460
:104DF000F4228091E10084FF30C08091E20084FFC2
:104E00002CC080E189BD82E189BD09B400FEFDCFDF
:104E10008091D8008F7D8093D8008091E1008F7EB3
:104E20008093E1008091E2008F7E8093E200809188
:104E3000E20081608093E2008091A003882311F05A
:104E400084E007C08091E30087FD02C081E001C0DB
:104E500083E08093A4030E94FC228091E10083FF01
:104E600029C08091E20083FF25C08091E100877F07
:104E70008093E10082E08093A4031092A0038091CC
:104E8000E1008E7F8093E1008091E2008E7F80932D
:104E9000E2008091E20080618093E20042E060E005
:104EA00080E00E9497258091F00088608093F00058
:104EB0000E94F222FF91EF91BF91AF919F918F914C
:104EC0007F916F915F914F913F912F910F900FBE06
:104ED0000F901F9018951F920F920FB60F921124EA
:104EE0002F933F934F935F936F937F938F939F93F2
:104EF000AF93BF93CF93DF93EF93FF93C091E900FC
:104F0000CF708091EC00D82FD17080FDD0E8109246
:104F1000E9008091F000877F8093F00078940E94F0
:104F2000AF271092E9008091F00088608093F00034
:104F3000CD2BCF70C093E900FF91EF91DF91CF911E
:104F4000BF91AF919F918F917F916F915F914F91A1
:104F50003F912F910F900FBE0F901F9018951F93A8
:104F6000CF93DF93CDB7DEB7AA970FB6F894DEBF25
:104F70000FBECDBFE5EAF3E08091F100819323E01D
:104F8000ED3AF207C9F70E941A238091E80083FFE7
:104F90002EC18091A5039091A603492F50E04A307D
:104FA000510508F024C1FA01EE59FF4F0C948329F2
:104FB000803821F0823809F01AC108C08091A1031D
:104FC0009091A203992389F082600FC08091A90378
:104FD0008F70873008F00BC18093E9008091EB005F
:104FE00085FB882780F91092E9009091E800977F6F
:104FF0009093E8008093F1001092F100D1C0282F27
:105000002D7F09F0F4C0882319F0823061F0EFC0E1
:105010008091A703813009F0EAC0933009F080E065
:105020008093A2032EC08091A70381112AC0809192
:10503000A9038F702FEF280F263008F0D8C0809377
:10504000E9002091EB0020FF1CC0933021F48091F7
:10505000EB00806214C09091EB0090619093EB00A4
:1050600021E030E0A90102C0440F551F8A95E2F704
:105070004093EA001092EA008091EB0088608093F0
:10508000EB001092E9008091E800877F8093E800B0
:105090000E94CC25ACC08111AAC01091A7031F7734
:1050A0008091E3008078812B8093E3008091E80079
:1050B000877F8093E8000E94CC258091E80080FFE4
:1050C000FCCF8091E30080688093E300111102C05F
:1050D00082E001C083E08093A40389C080588230BD
:1050E00008F085C08091A7039091A8038C3D53E000
:1050F000950779F583E08A838AE289834FB7F8942C
:10510000DE01139620E03EE051E2E32FF0E0509301
:105110005700E49120FF03C0E295EF703F5FEF700E
:105120008E2F90E0EA3010F0C79601C0C0968D93A4
:105130009D932F5F243149F74FBF8091E800877F0F
:105140008093E8006AE270E0CE0101960E94D824C4
:1051500016C06091A9037091AA03AE014F5F5F4F23
:105160000E941C24BC01892B09F441C09091E800E5
:10517000977F9093E80089819A810E9436258091DB
:10518000E8008B778093E80032C0803881F5809109
:10519000E800877F8093E8008091A0038093F1006E
:1051A0008091E8008E7772CF811121C08091A70392
:1051B0009091A80399270297D4F48091E800877F03
:1051C0008093E8008091A7038093A0030E94CC25E0
:1051D0008091A003811106C08091E30087FD02C089
:1051E00081E001C084E08093A4030E9406238091A3
:1051F000E80083FF0AC08091E800877F8093E80081
:105200008091EB0080628093EB00AA960FB6F89431
:10521000DEBF0FBECDBFDF91CF911F9108950895DE
:10522000CF938091A4038823A1F0C091E900CF70AF
:105230009091EC00892F817090FD80E8C82B10922E
:10524000E9008091E80083FD0E94AF27CF70C093F2
:10525000E900CF91089587FB082E062687FD8195EA
:1052600067FD61950E94BA290EF4919507FC81951E
:105270000895AA1BBB1B51E107C0AA1FBB1FA6179D
:10528000B70710F0A61BB70B881F991F5A95A9F7EF
:1052900080959095BC01CD01089597FB072E16F4DB
:1052A000009407D077FD09D00E94392907FC05D06A
:1052B0003EF4909581959F4F0895709561957F4F2D
:1052C0000895A1E21A2EAA1BBB1BFD010DC0AA1F47
:1052D000BB1FEE1FFF1FA217B307E407F50720F05F
:1052E000A21BB30BE40BF50B661F771F881F991FDA
:1052F0001A9469F760957095809590959B01AC0123
:10530000BD01CF010895EE0FFF1F0590F491E02D30
:1053100009940E949129332312F48A1B9B0B0C944D
:10532000A229A29FB001B39FC001A39F700D811D50
:105330001124911DB29F700D811D1124911D08959E
:105340000E949129B7FF0895821B930B08950E9434
:105350009129A59F900DB49F900DA49F800D911D44
:1053600011240895B7FF0C94A7290E94A729821B36
:10537000930B0895991B79E004C0991F961708F0C4
:10538000961B881F7A95C9F780950895FC014150B6
:10539000504030F001900616D1F73197CF010895B3
:1053A000882799270895FB01DC0104C08D910190A5
:1053B000801921F441505040C8F7881B990B08957B
:1053C000F999FECF92BD81BDF89A992780B50895CD
:1053D000A6E1B0E044E050E00C941A2AA8E1B0E065
:1053E00042E050E00C941A2A262FF999FECF92BD84
:1053F00081BDF89A019700B4021639F01FBA20BD9A
:105400000FB6F894FA9AF99A0FBE08950396272FCB
:105410000E94F5290E94F429252F0E94F529242FA6
:105420000C94F5290196272F0E94F5290C94F42954
:10543000DC01CB01FC01F999FECF06C0F2BDE1BD54
:10544000F89A319600B40D9241505040B8F7089543
:04545000F894FFCFFE
:10545400C8007602280850011E0A14010101020046
:105464002900292901191A1B1C1D1E1F2021224A4B
:10547400226D224E22DD22D9224D2201E200E900D2
:10548400EA00B500B600B700CD008301CC008A0164
:1054940092019401210223022402250226022702FA
:1054A4002A02B300B4006F007000818283E200E935
:1054B40000EA00B500B600B700CD008301CC008A35
:1054C40001920194012102230224022502260227CB
:1054D400022A02B300B4006F007000818283349703
:1054E40096949593929190663635F4F0C6F1F5F65C
:1054F400F7333231000102020202060606090909E5
:105504000909090F0F0F0F0F0F1515151819191980
:0A5514001919191919191923240097
:00000001FF
